:1000000009C016C015C014C013C012C012C010C061
:100010000FC00EC011241FBECFE9CDBF10E0A0E677
:10002000B0E001C01D92A436B107E1F76FD07CC0EB
:10003000E7CF1F920F920FB60F9211242F933F9389
:100040004F935F938F939F93809163008F5F809313
:100050006300833108F44FC01092630086B350915F
:10006000620090E08071907024E0959587952A95C4
:10007000E1F7252F30E02170307040916100821748
:10008000930711F44F5F01C0415040936100552325
:1000900069F48091610090916000823011F49F5F5B
:1000A00001C09150909360001092610080916000B7
:1000B00089321CF088E28093600080916000883D66
:1000C0001CF488ED80936000809160008F310CF00B
:1000D000C39A87FDC398852F8F5F8093620082301B
:1000E00010F01092620080916200882311F482E186
:1000F00001C082E28FBD9F918F915F914F913F919F
:100100002F910F900FBE0F901F90189581B781BF50
:1001100082E18FBD81E083BF8FE986BF84E089BF24
:0C0120007894B99ABB9AFFCFF894FFCFF7
:00000001FF
